:04000000B601DE293E
:100008000800B616B61EB612B6190E28B615472041
:10001800031835280830A3005B20A20DA30B102875
:10002800B61E402065206120B61A35203A202208E5
:100038000310D929B616B61EB61236192828FE3965
:10004800B70036150310D929361A3028A6003616F7
:1000580047200318352826084E2003183528B61ED1
:10006800D9294020652036113612B6113A08840085
:1000780038088417800446283A088400380980051F
:100088008417800508003A20652040206120370841
:10009800B6190138A2000830A300A20D03183A20AF
:1000A800031C402065206120A30B51283A206520BD
:1000B8003A08840038080005FF3E3B0884003909E7
:1000C80043283B08840039083D2864007F20031832
:1000D8006928CE20A8010830A300CF207F2003186C
:1000E800A80AAB1EA801A20CA30B7128AB1AA21375
:1000F800CF20220808003A088400380884178004B2
:10010800841300052B1B3806FF3E0800A4002908AD
:100118000319D929D421A00025188317240884009D
:10012800200880008313A40AA9038B280408A600CA
:100138003A0884008030B7050830A7000310031878
:10014800B70AB420A60CA70BA3280000AB1A370CDB
:10015800B420DC210314B4202F08A3002E083C2966
:100168008413AB1FC328000838042B1F38068000EF
:10017800841700083804031C38068000CF280008BC
:100188003804031C38062B1B3806800084173809EE
:100198008005CF2837172B081F39003EA1002A08F1
:1001A8000E3E0318A10A371F49293713A000023051
:1001B8007C214929B71329080319B7170430A80067
:1001C800250EEB202508EB20240EEB2024080F3900
:1001D800F63E0318073E0A3EF128A000A8030319BB
:1001E800B71329080319FB28280203180800200858
:1001F800031DB713B71B0800303ED42901308A000D
:1002080028080739820701340234043408341034CA
:1002180020344034803483178001840AFF3E031D54
:100228001029D929210820040319A00A8030201A8E
:10023800A1062019A106A018A106210DA00DA10D47
:10024800D92903178D0083168C130C1483120C08FC
:10025800D92903178C0083168C130C1555308D0083
:10026800AA308D008C148C1837290C11D929A301B8
:10027800A200FF30A207031CA307031CD9290330DF
:10028800A100E63049213D29A101FC3EA000A109B9
:10029800031C5429FF300000A00703184F29A007AA
:1002A8006400A10F4E290800A8000221A001A101A5
:1002B800A81DA000A819A1002008D929A201A301FE
:1002C8006929A10CA00CA20DA30DFF3E03186529F6
:1002D8002308A1002208A000D9290310A00DA10D10
:1002E800FF3E031871292008D9290310A10CA00C7E
:1002F800FF3E031879292008D929A101A301A200EA
:1003080002309229A301A20003309229A301A2007E
:1003180001309229A301A20006309229A8002308DF
:100328002102031D992922082002043003180130F4
:10033800031902302805031DFF30D929A501A4019E
:100348001030A600210DA40DA50D2208A402230833
:10035800031C230FA5020318B8292208A4072308A1
:100368000318230FA5070310A00DA10DA60BA6299E
:100378002008D9291030A800A101A001A70CA60CBB
:10038800031CCC292208A00723080318230FA10760
:10039800A10CA00CA50CA40CA80BC2292408D929CF
:1003A800840031088A003008820083130313831203
:1003B800640008002030840060308A011021A030D9
:1003C800840050308A0110211030840060308A0186
:1003D8000F219030840060308A010F218316D601E6
:1003E800D50120308400603083128A011021A030AA
:1003F800840050308A0110211030840060308A0156
:100408000F219030840060308A010F218316073055
:100418009F00990183129801831602309800DE012B
:10042800DF01861006118801071087100711831253
:100438000711861001308A013B21861464308A0135
:100448003B218A150A122B2B0710831634088312B6
:1004580088008A110A12352A07148316360883126F
:10046800880087100000871407100800831643309F
:10047800B60083128A0130228316FF308800831267
:1004880007140611000008088316C4008312061515
:100498000710831688018312080083160130C500EF
:1004A80083128A110A12B322831626088312A00027
:1004B800831627088312A1000830A200A3018A012D
:1004C800A2212408B2002508B30032088A01582165
:1004D800B2002108B3003208A0003308A100083098
:1004E8008A0162218316C10083128A013A226400BC
:1004F80083164508003C8A110A128312031D8C2AB0
:10050800831644084104C30083128A110A12912AEF
:10051800831644084106C300831283164630B6008A
:1005280083128A01302283162008B40083128A01BC
:1005380028227D088316B40083128A012822831694
:100548004230B60083128A01302283164308B40071
:1005580083128A0128228316C50183120800831694
:1005680028088312A600831629088312A7002030C2
:10057800A200A3018A01BE218316AE0083122508BA
:100588008316AF0026088312A0008316270883125B
:10059800A1000830A200A3018A01A2218316AC00A1
:1005A800831221088316AD002E082C078312B2008F
:1005B80083162F080318013E2D078312B30000305D
:1005C8003207FB0010300318013E3307FC007C089B
:1005D800FD00FE017B088316A000A1014630B6008D
:1005E80083128A01302283162008B40083128A01FC
:1005F80028227D088316B40083128A012822080065
:1006080083164E084B07A600A701A70D4F084C07F5
:10061800A800A901A90D83128A01552283164E0844
:100628004B02A600A701031CA7034F084C07A8000C
:10063800A901A90D83128A01552283164B084E077A
:10064800A600A701A70D4F084C02A800A901031C8A
:10065800A90383128A01552283164E084B02A6006D
:10066800A701031CA7034F084C02A800A901031CFB
:10067800A90383128A01552283164F084B07A60047
:10068800A701A70D4E084C07A800A901A90D8312C0
:100698008A01552283164F084B02A600A701031CA6
:1006A800A7034C084E07A800A901A90D83128A01C7
:1006B800552283164B084F07A600A701A70D4E0821
:1006C8004C02A800A901031CA90383128A01552220
:1006D80083164F084B02A600A701031CA7034E0868
:1006E8004C02A800A901031CA90383128A01552200
:1006F80008008316CE014D08CF0083120230A600F1
:10070800A70183164D088312A200A3018A01BE2106
:10071800B2002508B3003208023C8316AA008312EF
:100728003308031C013E003C8316AB0083126400AF
:1007380083164E084F028A110A128312031CF62BE5
:100748008A01042364008A110A1283168310AB1FDE
:10075800831483128318CE2B0430A600A7018316B6
:100768004E088312A200A3018A01BE21B200250807
:10077800B3000630B2070318B30A32088316AA0773
:10078800831233080318013E8316AB0783128A11BC
:100798000A12F12B83164F084E028312B200B301DE
:1007A800031CB3030430A600A7013208A2003308D3
:1007B800A3008A01BE21B2002508B3000A30B2079F
:1007C8000318B30A32088316AA07831233080318DA
:1007D800013E8316AB07CF0383128316CE0A83121A
:1007E8008A019B2B08008316CE014D08CF00831287
:1007F8000230A600A70183164D088312A200A301A8
:100808008A01BE21B2002508B3003208023C8316D3
:10081800AA0083123308031C013E003C8316AB0078
:100828008312640083164E084F028A110A1283123B
:10083800031C3E2C8A0104230430A600A70183165A
:100848004E088312A200A3018A01BE21B200250826
:10085800B3000630B2070318B30A32088316AA0792
:10086800831233080318013E8316AB07CE0A83129E
:100878008A01152C08008316CE014D08CF0083127B
:100888000230A600A70183164D088312A200A30117
:100898008A01BE21B2002508B3003208023C831643
:1008A800AA0083123308031C013E003C8316AB00E8
:1008B8008312640083164E084F028A110A128312AB
:1008C800031C8F2C8A01042383164F084E028312BF
:1008D800B200B301031CB3030430A600A701320819
:1008E800A2003308A3008A01BE21B2002508B30084
:1008F8000A30B2070318B30A32088316AA0783120C
:1009080033080318013E8316AB070330CF02CE0A23
:1009180083128A015D2C08008316CE014D08CF0092
:1009280083120230A600A70183164D088312A20085
:10093800A3018A01BE21B2002508B3003208023C97
:100948008316AA0083123308031C013E003C831659
:10095800AB008312640083164E084F028A110A12F4
:100968008312031CDF2C8A01042383164F084E02CE
:100978008312B200B301031CB3030430A600A7011D
:100988003208A2003308A3008A01BE21B20025085C
:10099800B3000A30B2070318B30A32088316AA074D
:1009A800831233080318013E8316AB07CF03CE0A20
:1009B80083128A01AE2C08008A110A1218258316A0
:1009C8004608BA008312640083163A0847028A115F
:1009D8000A128312031C172D83164908BD008312BF
:1009E800640083163D084A028A110A128312031C06
:1009F8000F2D83163A08A600A7013D08A800A901F3
:100A080083128A01552283165908BD078A110A12D2
:100A18008312031CF42C83165908BA078A110A1288
:100A28008312031CE72C080064008316460847025B
:100A38008A110A1283120318272D831646084702C3
:100A4800C607C70283126400831649084A028A113E
:100A58000A1283120318362D831649084A02C90759
:100A6800CA028312080083165B08A600A7015D0866
:100A7800A800A9018312831628088312A0008316F0
:100A880029088312A10083165C0883128A018A212F
:100A98008A110A12031D5B2D8A0155228316A80AA2
:100AA8000319A90A8A110A128312031D3F2D013066
:100AB80083165B07A600A701A70D5D08A800A9017A
:100AC8008312831628088312A0008316290883122C
:100AD800A10083165C0883128A018A218A110A12EE
:100AE800031D872D8A01552283165908A8078A11E4
:100AF8000A128312031C652D8316A80A8A110A128A
:100B08008312031D652D080083165D08A800A9013E
:100B18005B08A600A7018312831626088312A0008B
:100B2800831627088312A10083165A0883128A01A4
:100B38008A218A110A12031DAC2D8A0155228316B7
:100B4800A60A0319A70A8A110A128312031D902DF7
:100B5800FF3083165D07A800FF300318013EA90087
:100B68005B08A600A7018312831626088312A0003B
:100B7800831627088312A10083165A0883128A0154
:100B88008A218A110A12031DDA2D8A015522831639
:100B98005908A6078A110A128312031CB82D831656
:100BA800A60A8A110A128312031DB82D08008A01A9
:100BB8001825831646084702BF0049084A02C000A4
:100BC800640040083F028A110A128312031C6A2E2D
:100BD800831640088312A000A10102308A01742103
:100BE800B2002108B30083163F088312320283162D
:100BF800AA0083123308031CFF3E8316AB00490882
:100C0800A800A9014608A600A70183128316260892
:100C18008312A000831627088312A10083164708B1
:100C280083128A018A218A110A12031D692E64001F
:100C38008A110A1283168310AB1F83148312831838
:100C48003D2E831640088312A000A10102308A01BC
:100C58007421B2002108B30032088316AA07831250
:100C680033080318013E8316AB0783128A110A1250
:100C78005E2E83163F0840028312B200B301031CA4
:100C8800B3030230A600A7013208A2003308A3006C
:100C98008A01BE21B2002508B30032088316AA07CC
:100CA800831233080318013E8316AB07A80A0319F9
:100CB800A90A83128A0155228316A60A0319A70ACC
:100CC8008A110A128312031D0A2E080083163F0890
:100CD8008312A000A10102308A017421B200210808
:100CE800B30083164008831232028316AA008312C7
:100CF8003308031CFF3E8316AB004608A600A70175
:100D08004908A800A9018312831628088312A000A5
:100D1800831629088312A10083164A0883128A01C0
:100D28008A218A110A12031DE72E64008A110A1209
:100D380083168310AB1F831483128318BB2E83166C
:100D48003F088312A000A10102308A017421B20079
:100D58002108B30032088316AA0783123308031840
:100D6800013E8316AB0783128A110A12DC2E831602
:100D780040083F028312B200B301031CB3030230E0
:100D8800A600A7013208A2003308A3008A01BE21E9
:100D9800B2002508B30032088316AA078312330865
:100DA8000318013E8316AB07A60A0319A70A831284
:100DB8008A0155228316A80A0319A90A8A110A1258
:100DC8008312031D882E08008A01182583164608F9
:100DD800BA008312640083163A0847028A110A127D
:100DE8008312031C102F83163A08A600A70149088E
:100DF800A800A90183128A01552283164A08A8006F
:100E0800A90183128A01552283165908BA078A1143
:100E18000A128312031CEE2E83164908BA008312A5
:100E2800640083163A084A028A110A128312031CC4
:100E3800362F83163A08A800A9014608A600A7017C
:100E480083128A01552283164708A600A701831238
:100E58008A01552283165908BA078A110A12831281
:100E6800031C142F080083164630B60083128A012B
:100E780030228316B40183128A0128228316103087
:100E8800B40083128A01282283164C30B6008312DC
:100E98008A01302283164230B60083128A0130223A
:100EA80083160130BA0083126400813083163A0237
:100EB8008A110A1283120318812F83160130BD008C
:100EC80083126400213083163D028A110A128312AC
:100ED80003187A2F8316B40183128A0128228316F5
:100EE800BD0A8A110A128312031D652F8316BA0AD6
:100EF8008A110A128312031D582F080083164630E0
:100F0800B60083128A0130228316B40183128A0143
:100F1800282283161030B40083128A012822080080
:100F280083164630B60083128A0130228316B40134
:100F380083128A0128228316B40183128A01282287
:100F480083164C30B60083128A0130228316423051
:100F5800B60083128A01302283160130BA00831248
:100F68006400113083163A028A110A128312031898
:100F7800DE2F83160130BD008312640021308316F2
:100F88003D028A110A1283120318D72F83162030C4
:100F9800B40083128A0128228316BD0A8A110A1214
:100FA8008312031DC12F8316BA0A8A110A128312EB
:100FB800031DB42F080083164630B60083128A0139
:100FC80030228316B40183128A0128228316B401C1
:100FD800831208008A0137278A0182278A01942709
:100FE8008A01DF27080083164030B60083128A0181
:100FF80030228316BA0183126400083083163A023D
:101008008A150A1283120318312883163A08073CF6
:101018008A150A128312031C28288A150A121A2014
:101028008316B40083128A150A12282808308A0009
:1010380083163A08831282073034873407341F3402
:1010480052347F34203400348A0128228316BA0AA5
:101058008A150A128312031D002883164430B6002D
:1010680083128A0130228316BA0183126400063083
:1010780083163A028A150A128312031869288316FE
:101088003A08053C8A150A128312031C60288A153F
:101098000A1254208316B40083128A150A12602893
:1010A80008308A0083163A08831282070034003415
:1010B8007F34003410347F348A0128228316BA0A18
:1010C8008A150A128312031D3A2883165A30B6006D
:1010D80083128A0130228316B40183128A012822DE
:1010E80083165B30B60083128A01302283160130E2
:1010F800B40083128A01282283165830B60083125E
:101108008A01302283161630B40083128A012822FD
:101118008A0137278A01942783164630B60083123E
:101128008A0130228316B40183128A012822831689
:10113800B40183128A01282283164C30B600831228
:101148008A01302283164230B40083128A01282291
:101158008316B40183128A01282283165D30B600F3
:1011680083128A01302283160430B40083128A0164
:10117800282283168630B40083128A012822831617
:101188005930B60083128A01302283161430B40015
:1011980083128A01282283164C30B60083128A01F2
:1011A8003022080083164630B60083128A013022A6
:1011B8007B088316B40083128A0128227C088316D0
:1011C800B40083128A01282283163708B6008312D6
:1011D8008A013022080083163A085C3E8400000821
:1011E8008312B200FF30A200A20A22080F3C8A151F
:1011F8000A12031C22298A150A120E2132028A15A4
:101208000A12031DF82822088316D20083128A15B1
:101218000A12222909308A00220882073034313420
:10122800323433343434353436343734383439346A
:1012380061346234633464346534663408002030C1
:10124800A600A701831628088312A200831629087E
:101258008312A3008A01BE21B2002508B300320818
:10126800A0003308A1000830A200A3018A01A2212E
:10127800B2002108B300831626088312A000831643
:1012880027088312A1000830A200A3018A01A22125
:10129800B4002108B50032083407FB0033080318EE
:1012A800013E3507FC008A150A1288292030A6005D
:1012B800A701831628088312A2008316290883121F
:1012C800A3008A01BE21B2002508B30083162608B0
:1012D8008312A000831627088312A1000830A200F9
:1012E800A3018A01A221B4002108B5003208B4077D
:1012F80033080318013EB50700303407FB001030EF
:101308000318013E3507FC008A150A12D6208316F9
:101318004230B60083128A01302283163508B400A1
:1013280083128A01282208000730BA004030B8002A
:101338002030AA00AB01AE01AF010230A90083162C
:1013480035088312A400A5019A30B000B1018A01C2
:10135800DE2008000730BA008030B8002030AA002C
:10136800AB018A0169205D3C8A150A12031DB52963
:101378000230A9006930B000B101A5015C308A01D2
:101388008A208316BA0183126400023083163A0257
:101398008A150A1283120318E0298A150A12EF2007
:1013A80083163A085C3E840052088000BA0A8A15FF
:1013B8000A128312031DC8295C08A000A101043089
:1013C8008A017421B2002108B3005D083204FF00CD
:1013D80008000730BA008030B8002030AA00AB01FE
:1013E8008A0169205D3C8A150A12031DF42904301C
:1013F800A9006930B000B101A5015C308A018A20DA
:101408008316BA0183126400043083163A028A15DF
:101418000A12831203181F2A8A150A12EF2083164C
:101428003A085C3E840052088000BA0A8A150A12FB
:101438008312031D072A5C08A000A10104308A0159
:101448007421B2002108B3005D083204FF005E0871
:10145800A000A10104308A017421B2002108B30060
:101468005F0832048316B000831208000730BA0000
:101478008030B8002030AA00AB018A0169205D3CA9
:101488008A150A12031D412A0630A9006930B000E6
:10149800B101A5015C308A018A208316BA01831242
:1014A8006400063083163A028A150A12831203185A
:1014B8006C2A8A150A12EF2083163A085C3E8400CB
:1014C80052088000BA0A8A150A128312031D542A88
:1014D8005C08A000A10104308A017421B20021082F
:1014E800B3005D083204FF005E08A000A1010430CB
:1014F8008A017421B2002108B3005F083204831600
:10150800B00083126008A000A10104308A01742190
:10151800B2002108B300610832048316B1008312B7
:1015280008000730BA008030B8002030AA00AB01AC
:101538008A0169205D3C8A150A12031D9C2A8A01CA
:1015480069208316D20030305202D9005208B50003
:10155800831208000730BA008030B8002030AA0093
:10156800AB018A0169205D3C8A150A12031DB52A60
:101578000830A9006930B000B101A5015C308A01CA
:101588008A208316BA0183126400083083163A024F
:101598008A150A1283120318E02A8A150A12EF2004
:1015A80083163A085C3E840052088000BA0A8A15FD
:1015B8000A128312031DC82A5C08A000A101043086
:1015C8008A017421B2002108B3005D083204831631
:1015D800C60083125E08A000A10104308A017421AC
:1015E800B2002108B3005F0832048316C7008312D3
:1015F8006008A000A10104308A017421B20021080A
:10160800B300610832048316C90083126208A0007F
:10161800A10104308A017421B2002108B3006308D3
:1016280032048316CA00831208007F088316CB0091
:101638003008CC003108CD00831208007F088316DB
:10164800A600A7013008A800A901831208008A0192
:10165800F7278A01EE27C530FB00FC0183164C30C2
:10166800B70083128A150A12D62083164230B600B4
:1016780083128A0130228316BA018312640016305D
:1016880083163A028A150A1283120318812B8316CD
:101698003A08153C8A150A128312031C782B8A15FE
:1016A8000A125C238316B40083128A150A12782B57
:1016B8000B308A0083163A08831282075034493463
:1016C8004334203443346F346E34743472346F349A
:1016D8006C346C34653464342034533445344434C5
:1016E80031343334333430348A0128228316BA0A29
:1016F8008A150A128312031D422BE330FB00FC01FA
:1017080083164C30B70083128A150A12D620831626
:101718004230B60083128A0130228316BA0183123E
:1017280064001B3083163A028A150A1283120318C2
:10173800D82B83163A081A3C8A150A128312031CFE
:10174800CF2B8A150A12AE238316B40083128A158A
:101758000A12CF2B0B308A0083163A0883128207AD
:101768005534733469346E346734203450346934F2
:1017780063344234613473346934633450347234BA
:101788006F3420345634653472342E342034323475
:101798002E34333432348A0128228316BA0A8A1541
:1017A8000A128312031D942B0530FB000130FC0044
:1017B80083164C30B70083128A150A12D620831676
:1017C8004230B60083128A0130228316BA0183128E
:1017D8006400153083163A028A150A128312031818
:1017E8002A2C83163A08143C8A150A128312031C01
:1017F800212C8A150A1206248316B40083128A152E
:101808000A12212C0C308A0083163A0883128207A8
:10181800523461346E346A34693474342034443454
:1018280069346F346C3420342D34203443344F34CD
:101838004D3450345334793473348A012822831652
:10184800BA0A8A150A128312031DEC2B2430FB00F6
:101858000130FC0083164C30B70083128A150A1237
:10186800D62083164230B60083128A0130228316AE
:10187800BA0183126400173083163A028A150A12D5
:10188800831203187E2C83163A08163C8A150A120E
:101898008312031C752C8A150A1258248316B40067
:1018A80083128A150A12752C0C308A0083163A089E
:1018B8008312820768347434743470343A342F34A1
:1018C8002F347734773477342E3463346F346D346F
:1018D800703473347934733431342E3463346F3460
:1018E8006D348A0128228316BA0A8A150A128312CD
:1018F800031D3E2C8316C601C901FF30C7007F3087
:10190800CA000130D90083128A01E8268316043000
:10191800C6000430C900FB30C7007B30CA00831200
:101928008A01E8260F30A300A0308A013C218A01F1
:10193800EE270530FB00FC0183164C30B7008312FC
:101948008A150A12D62083164230B60083128A01FD
:1019580030228316BA0183126400143083163A02C7
:101968008A150A1283120318ED2C83163A08133CC1
:101978008A150A128312031CE42C8A150A12CA2437
:101988008316B40083128A150A12E42C0C308A00DC
:1019980083163A0883128207443452344134573448
:1019A8002034473452344134503448344934433471
:1019B8002034443445345334493447344E34533452
:1019C8008A0128228316BA0A8A150A128312031D6D
:1019D800B02C83162330CB004030CC000A30CD0029
:1019E800831264001F3083164D028A150A1283126F
:1019F8000318082D8A017D230A308316CD078A151E
:101A08000A128312031CF52C83166430CB00403075
:101A1800CC000A30CD00831264001F3083164D02BB
:101A28008A150A1283120318232D8A01F7230A3014
:101A38008316CD078A150A128312031C102D8316EC
:101A4800A030CB004030CC000A30CD0083126400B7
:101A58001F3083164D028A150A12831203183E2D71
:101A68008A0190240A308316CD078A150A12831238
:101A7800031C2B2D8316DC30CB004030CC000A3001
:101A8800CD00831264001F3083164D028A150A1296
:101A980083120318592D8A013F240A308316CD0773
:101AA8008A150A128312031C462D0F30A300A0309A
:101AB8008A013C218A01EE27C530FB00FC01831610
:101AC8004C30B70083128A150A12D620831642308A
:101AD800B60083128A0130228316BA018312640089
:101AE800133083163A028A150A1283120318AF2D8F
:101AF80083163A08123C8A150A128312031CA62D73
:101B08008A150A128D258316B40083128A150A12C3
:101B1800A62D0D308A0083163A08831282072034D6
:101B280042347934203443344F344D3450345334B0
:101B380079347334283463342934203432343034DB
:101B4800303432348A0128228316BA0A8A150A12D6
:101B58008312031D732D0B30A300B8308A013C217A
:101B68008A01EE2783161030DB000430D9002030BC
:101B7800DD006E30DC0083128A01372583166E3053
:101B8800DD007830DA0083128A0188256430FB0092
:101B9800FC0183164C30B70083128A150A12D6202E
:101BA80083164230B60083128A0130228316BA01A6
:101BB800831264000A3083163A028A150A128312C5
:101BC8000318142E83163A08093C8A150A12831240
:101BD800031C0B2E8A150A12F7258316B4008312EC
:101BE8008A150A120B2E0E308A0083163A088312C1
:021BF800002EBD
:101C00008207533459345334543445344D342034DA
:101C10004C344F3447348A0128228316BA0A8A1575
:101C20000A128312031DDD2DA030FB00FC01831678
:101C30004F30B70083128A150A12D620831642301D
:101C4000B60083128A0130228316BA01831264001F
:101C5000083083163A028A150A1283120318582E86
:101C600083163A08073C8A150A128312031C4F2E6A
:101C70008A150A1241268316B40083128A150A12A5
:101C80004F2E0E308A0083163A08831282074134A1
:101C900043345434493456344934543459348A0121
:101CA00028228316BA0A8A150A128312031D272EC8
:101CB0008130FB00FC0183164F30B70083128A1578
:101CC0000A12D62083164230B60083128A013022CF
:101CD0008316BA01831264000A3083163A028A1509
:101CE0000A12831203189E2E83163A08093C8A159D
:101CF0000A128312031C952E8A150A128526831652
:101D0000B40083128A150A12952E0E308A008316AB
:101D10003A0883128207393438343734363435344C
:101D2000343433343234313430348A012822831647
:101D3000BA0A8A150A128312031D6B2EE330FB00C8
:101D40000130FC0083164C30B70083128A150A124A
:101D5000D62083164230B60083128A0130228316C1
:101D6000BA0183126400063083163A028A150A12F9
:101D700083120318E12E83163A08053C8A150A12CD
:101D80008312031CD82E8A150A12CC268316B4009F
:101D900083128A150A12D82E0E308A0083163A084A
:101DA0008312820748344F34553452344C345934FA
:101DB0008A0128228316BA0A8A150A128312031D81
:101DC000B22E83161030DB007830DA002030DD00D0
:101DD0006E30DC005C08A800A9015B08A600A70122
:101DE0008312831626088312A00083162708831205
:101DF000A10083165A0883128A018A218A150A12C1
:101E0000031D682F831622088312A000831623085F
:101E10008312A1008A01162120088316A2008312D2
:101E200021088316A3006400803022028A150A125A
:101E30008312031C262F01308316A8020030031CD6
:101E4000013EA90283128A150A122B2F8316A80AB3
:101E50000319A90A8312831628088312A000831687
:101E600029088312A10083165C0883128A018E213F
:101E70008A150A12031D452FFF3083165C07A80040
:101E8000FF300318013EA90083128316280883122D
:101E9000A000831629088312A10083165D0883120F
:101EA0008A0186218A150A12031D5D2F01308316CF
:101EB0005D07A800A901A90D83128A015522831686
:101EC000A60A0319A70A8A150A128312031DF12E06
:101ED000F030FB00FC0183164C30B70083128A15EA
:101EE0000A12D62083164230B60083128A013022AD
:101EF0008316BA01831264000D3083163A028A15E4
:101F00000A1283120318B12F83163A080C3C8A1563
:101F10000A128312031CA82F8A150A12952783160A
:101F2000B40083128A150A12A82F0F308A00831674
:101F30003A08831282075434653472346D3469343C
:101F40006E3461346C3420344D346F346434653411
:101F50008A0128228316BA0A8A150A128312031DDF
:101F60007B2F1030FB000130FC0083164C30B70093
:101F700083128A150A12D62083164230B6008312C5
:101F80008A0130228316BA01831264000D30831651
:101F90003A028A150A1283120318FB2F83163A0895
:101FA0000C3C8A150A128312031CF22F8A150A129E
:101FB000DF278316B40083128A150A12F22F0F301E
:101FC0008A0083163A0883128207573461346934D1
:101FD000743469346E3467342E342E342E342E34F7
:101FE0002E342E348A0128228316BA0A8A150A1240
:101FF0008312031DC52F5030FB000130FC008316F7
:102000004C30B70083128A150A12D620831642304C
:10201000B60083128A0130228316BA01831264004B
:102020000E3083163A028A110A16831203184628C4
:1020300083163A080D3C8A110A168312031C3D28A8
:102040008A110A1629208316B40083128A110A16EF
:102050003D2810308A0083163A08831282075534CF
:1020600073346534203447344C3455345434493453
:102070004C34203431342E3433348A0128228316F0
:10208000BA0A8A110A168312031D0F280730BA00F4
:102090004030B8002030AA00AB01AE01AF01523091
:1020A0008A019B2065308A019B2061308A019B2038
:1020B00064308A019B2079308A019B203A308A0162
:1020C0009B200A308A019B200D308A019B2007301B
:1020D000BA008030B8002030AA00AB018A01692024
:1020E0005D3C8A110A16031D6E288A016920831639
:1020F000D20052088312A00063308A018121B2000D
:10210000831652088312A00043308A018121B40053
:10211000320834048A110A16031D752A83165208E0
:102120008312A00073308A018121B2008316520805
:102130008312A00053308A018121B4003208340494
:102140008A110A16031D802A831652088312A000E2
:1021500071308A018121B200831652088312A000D7
:1021600051308A018121B400320834048A110A16E0
:10217000031D8B2A831652088312A00074308A0133
:102180008121B200831652088312A00054308A01C4
:102190008121B400320834048A110A16031D962ADC
:1021A000831652088312A0006C308A018121B2008C
:1021B000831652088312A0004C308A018121B4009A
:1021C000320834048A110A16031DB72A83165208EE
:1021D0008312A00072308A018121B2008316520856
:1021E0008312A00052308A018121B40032083404E5
:1021F0008A110A16031DAC2A831652088312A00006
:1022000062308A018121B200831652088312A00035
:1022100042308A018121B400320834048A110A163E
:10222000031DA12A831652088312A0006B308A0175
:102230008121B200831652088312A0004B308A011C
:102240008121B400320834048A110A16031DE52ADC
:10225000831652088312A00064308A018121B200E3
:10226000831652088312A00044308A018121B400F1
:10227000320834048A110A16031DEE2A8316520806
:102280008312A00065308A018121B20083165208B2
:102290008312A00045308A018121B4003208340441
:1022A0008A110A16031DEA2A831652088312A00017
:1022B00070308A018121B200831652088312A00077
:1022C00050308A018121B400320834048A110A1680
:1022D000031DFC2A831652088312A00075308A0160
:1022E0008121B200831652088312A00055308A0162
:1022F0008121B400320834048A110A16031D0F2B01
:10230000831652088312A00078308A018121B2001E
:10231000831652088312A00058308A018121B4002C
:10232000320834048A110A16031DBF2A8316520884
:102330008312A00079308A018121B20083165208ED
:102340008312A00059308A018121B400320834047C
:102350008A110A16031DD22A831652088312A0007E
:1023600066308A018121B200831652088312A000D0
:1023700046308A018121B400320834048A110A16D9
:10238000031D1F2B831652088312A00068308A0198
:102390008121B200831652088312A00048308A01BE
:1023A0008121B400320834048A110A16031D2F2B30
:1023B000831652088312A00076308A018121B20070
:1023C000831652088312A00056308A018121B4007E
:1023D000320834048A110A16031D842B831652080E
:1023E0008312A0006D308A018121B2008316520849
:1023F0008312A0004D308A018121B40032083404D8
:102400008A110A16031D0C2D831652088312A00090
:102410006E308A018121B200831652088312A00017
:102420004E308A018121B400320834048A110A1620
:10243000031D8E2C831652088312A0006F308A0170
:102440008121B200831652088312A0004F308A0106
:102450008121B400320834048A110A16031DE92BC5
:10246000831652088312A00061308A018121B200D4
:10247000831652088312A00041308A018121B400E2
:10248000320834048A110A16031DEF2B83165208F2
:102490008312A00067308A018121B200831652089E
:1024A0008312A00047308A018121B400320834042D
:1024B0008A110A16031DE22B831652088312A0000C
:1024C00077308A018121B200831652088312A0005E
:1024D00057308A018121B400320834048A110A1667
:1024E000031DDB2B8A110A1646288A150A123A2286
:1024F0008A150A1219238A017D238A110A16462891
:102500008A150A123A228A150A1219238A01F72318
:102510008A110A1646288A150A123A228A150A12C0
:1025200019238A0190248A110A1646288A150A124C
:102530003A228A150A1219238A013F248A110A169F
:1025400046288A150A12AE228A150A1295228A0195
:10255000E0248A110A1646288A150A12AE228A1524
:102560000A1295228A01E8268A110A1646288A1537
:102570000A12AE228A01DB258A110A1646288A151C
:102580000A123A227F088316DB003008DA0031088D
:10259000DD0083128A150A1295228A0188258A1184
:1025A0000A1646288A150A123A227F088316DD0089
:1025B0003008DC003108DB0083128A150A129522EC
:1025C0008A0137258A110A1646288A01EE278A11C0
:1025D0000A16462883160130C50083128A150A128E
:1025E000ED218A150A1222238A0155228316C5017C
:1025F00083128A110A16462883164C30B7008312BC
:102600008A150A12ED218A150A1222238A150A1246
:1026100095228A150A1223218A110A1646288A153C
:102620000A123A228A150A12222383163108B500AB
:1026300083128A150A125A218A110A1646288A1507
:102640000A1295228316C601FF30C700C9017F30E8
:10265000CA0083128A01E0248A110A1646288316CA
:102660004C30B70083128A150A12ED218A150A121E
:10267000222383164808DE0083128A150A12952247
:10268000640083163508403C8A110A168312031928
:10269000812B6400831635083B3C8A110A1683128D
:1026A000031D5C2B83162030B50083128A150A1295
:1026B00023218A110A16632B83163508B30083126F
:1026C0008A150A12232108308316A6070318A70AC1
:1026D00026088312A000831627088312A100A301F5
:1026E000EF308A018F218A110A16031D7B2B831676
:1026F0005E08C80083128A150A1295228A110A16EA
:10270000402B8A110A16462883164D30B7008312D3
:102710008A150A12ED218A150A1222238316260829
:10272000DE002808DF0083128A150A129522640051
:1027300083163508403C8A110A1683120319D82BD8
:102740006400831635083B3C8A110A168312031D68
:10275000B32B83162030B50083128A150A12232169
:102760008A110A16B62B8A150A12232183165E08CF
:10277000A600A7010830A8070318A90A2808831291
:10278000A000831629088312A100A3017F308A01CB
:102790008F218A110A16031DD22B83165F08A80009
:1027A000A90183128A150A1295228A110A16972BFB
:1027B0008A110A16462883160230B90083128A113C
:1027C0000A16F32B83160330B90083128A110A16F6
:1027D000F32B8316B90183128A110A16F32B831681
:1027E0000130B90083128A150A12AE2283164608F8
:1027F0008312F600831647088312F50083164908F2
:102800008312F80083164A088312F7007508F30054
:102810007608F4007308A0007408A1007808A300EB
:1028200077088A018B218A110A16031D882C6400FF
:1028300083163908003C8A110A168312031D3A2CAC
:102840008A150A12AE210730BA001030B8000730DE
:10285000BB000830B900A0308A01202074088A012A
:10286000202073088A0120207F088A011E200A3058
:102870008A013B21640083163908013C8A110A163B
:102880008312031D5C2C0730BA001030B8000730EB
:10289000BB000830B900A0308A01202074088A01EA
:1028A000202073088A0120208A0105208316B500A4
:1028B00083128A150A129821640083163908023C93
:1028C0008A110A168312031D6F2C8A150A12AE2173
:1028D000730803178D0003137F088A012D216400FC
:1028E00083163908033C8A110A168312031D812CB2
:1028F00073088A0125218316B50083128A150A12EE
:102900009821F30A0319F40A8A110A16031D0A2CE6
:102910008316B90183128A110A1646288A150A12EB
:10292000AE2283164908A800A9018312831628083D
:102930008312A000831629088312A10083164A0877
:1029400083128A018A218A110A16031D092D831612
:102950004608A600A7018312831626088312A0004A
:10296000831627088312A1008316470883128A0161
:102970008A218A110A16031D002D2030A600A70106
:10298000831628088312A200831629088312A30045
:102990008A01BE21B2002508B300831626088312DF
:1029A000A000831627088312A1000830A200A3010B
:1029B0008A01A221B4002108B5003208B407330807
:1029C0000318013EB50700303407FB001030031830
:1029D000013E3507FC008A150A12D6208A013A22E8
:1029E00083164408B50083128A150A1298218316AB
:1029F000A60A0319A70A8A110A168312031DAC2C12
:102A00008316A80A0319A90A8A110A168312031D3C
:102A1000962C8A110A1646288A150A12AE228316A7
:102A20004908A800A9018312831628088312A00070
:102A3000831629088312A10083164A0883128A018B
:102A40008A218A110A16031D572D83164608A600EF
:102A5000A7018312831626088312A0008316270875
:102A60008312A1008316470883128A018A218A11E2
:102A70000A16031D4E2D8A150A12AE217F088316F1
:102A8000B40083128A150A125A218316A60A031962
:102A9000A70A8A110A168312031D2A2D8316A80A73
:102AA0000319A90A8A110A168312031D142D630043
:062AB0008A110A16572DE1
:02400E00753DFE
:00000001FF
